:1000000019C033C032C031C030C02FC02EC02DC087
:100010002CC02BC02AC029C028C027C026C025C09C
:1000200024C023C022C021C020C01FC01EC01DC0CC
:100030001CC01BC011241FBECFEFD4E0DEBFCDBF5C
:1000400011E0A0E0B1E0E8E9F0E002C005900D9217
:10005000A030B107D9F711E0A0E0B1E001C01D92D6
:10006000A030B107E1F702D015C0CACF239A29E129
:1000700030E02B9A80E197E2F9013197F1F701978F
:10008000D9F72B9880E49CE9F9013197F1F70197B2
:08009000D9F7EFCFF894FFCF80
:00000001FF
